:020000040000FA
:10000000C0B6D1C0C1C4CCEC0000000000000000AC
:1000100000000000030000000002000014000000C7
:10002000016070474DF6793CC0F60D0C604744F610
:10003000196CC0F6020C604741F2DF5CC0F60D0C93
:10004000604747F6AF5CC0F60E0C604744F6935C21
:10005000C0F6020C60474EF6F95CC0F60D0C604726
:100060004BF6676CC0F60D0C60474EF6DB7CC0F6B5
:100070000D0C60474EF61B2CC0F60D0C604747F682
:10008000E34CC0F60E0C60474FF2753CC0F60D0C09
:1000900060474CF2131CC0F60D0C60474CF2AD1CCF
:1000A000C0F60D0C60474BF6911CC0F60D0C604776
:1000B00048F6ED2CC0F60D0C60474CF2591CC0F60A
:1000C0000E0C604741F2136CC0F60D0C60474EF207
:1000D000417CC0F60D0C60474FF23B3CC0F60D0C66
:1000E00060474DF6273CC0F60D0C604748F67F3C54
:1000F000C0F60D0C604748F2110CC0F60D0C6047BD
:1001000044F6B91CC0F6020C60474FF68D3CC0F6B1
:100110000D0C60474AF25D2CC0F60D0C604748F2AA
:10012000553CC0F60D0C604747F6E34CC0F60E0C8C
:10013000604747F6315CC0F60E0C604744F6817CA0
:10014000C0F6020C60474DF2DF5CC0F6020C60475F
:100150004BF2590CC0F6020C60474BF2610CC0F632
:10016000020C604745F6137CC0F6020C604745F66A
:10017000C37CC0F6020C604745F6E72CC0F6020CC3
:10018000604745F6D11CC0F6020C604748F2912C3E
:10019000C0F6020C604748F25F3CC0F6020C6047B4
:1001A00048F26F4CC0F6020C604744F6E31CC0F600
:1001B0000D0C604748F2DB5CC0F6020C604745F26C
:1001C000EF7CC0F6020C604748F2C54CC0F6020C4A
:1001D000604748F2256CC0F6020C604744F6C72C15
:1001E000C0F6020C604740F2812CC0F6020C60475A
:1001F00040F2852CC0F6020C604748F6871CC0F61A
:100200000D0C604748F65D1CC0F60D0C604748F2C7
:10021000796CC0F60D0C60472DE9F04591B00446AD
:100220000E46D4F8B40DB04228D100200F901090A3
:10023000D4F8A41DD1F8F42004F5E47151F822009B
:100240000FA900F0B3FC0FA904F5337000F04FFDC7
:10025000012809D141F288306EA370A272A10090EA
:100260002046FFF7DFFE08E041F2883069A370A264
:100270006DA100902046FFF7D5FEC8E0D4F8BC0D74
:10028000B04235D10127D4F8C00D28B1D4F8C00D43
:10029000B0F8F400401C87B2D4F8B00D00F1F405BA
:1002A0004FF48070FFF7C3FE804641462846FFF7B3
:1002B000C3FE4046FFF7C5FE8246534642463946D6
:1002C00004F5337000F028FF4046FFF7BFFE02231D
:1002D0005AA2394604F5337000F01EFFD4F8B01D61
:1002E00001F1F4027321D4F8AC0DFFF7B4FE8EE0F7
:1002F000D4F8B80DB042C0D1D4F8C401022814D14A
:10030000D4F8A80D00F1F40104F5337000F06DFF8E
:10031000D4F8A80DD0F8D01088470020C4F8A80D54
:1003200004F5337000F07EFF13E0D4F8C401012817
:100330000FD104F6A4542068D0F8D01088470020CC
:1003400020602069D0F8D010884700202061A4F6F2
:10035000A454012104F5337000F013FFD4F8B80D54
:10036000D0F8D01088470020C4F8B80D32212046BC
:10037000FFF776FEA568E768C820A5F10A03052205
:10038000114600902046FFF770FEC4F8AC0D2820FF
:10039000A5F1A003CD22052100902046FFF76AFEBB
:1003A000C4F8B00D20222649794409A8FFF767FE5A
:1003B00009A80490801D05900CA80690801D079048
:1003C0000FA8089028206421CD22A5F19B03CDE938
:1003D00000210290052204A92046FFF755FEC4F82B
:1003E000C00D19203221A5F13702D223CDE900102A
:1003F00000212046FFF74DFEC4F8BC0D11A1D4F832
:10040000BC0DFFF74BFE2046FFF74DFE00BF11B0BD
:10041000BDE8F085C8B7B6A800000000C1ACBDD3E8
:10042000B3C9B9A600000000CCE1CABE00000000BC
:10043000C1ACBDD3CAA7B0DC000000000D0A0000AB
:1004400048150000B7A2CBCD000000002DE9F04117
:1004500006460C4601F07EF907464FF000080025DD
:1004600020680A2843D2DFE800F04209050D423037
:100470004222422C304600F0C1F839E0304600F00C
:100480003DF835E0E568287C00F0010000B900BFC8
:10049000287C00F0080020B13046D6F8D0108847FC
:1004A00026E0286910B13046FFF7FDFD20E0D4F8C2
:1004B0000C80D8F80800032800D100E000BF00BF7E
:1004C00016E0304600F028F812E0E068012802D07B
:1004D000022809D100E008E02069012803D1304654
:1004E0006168FFF799FE00E000BF00BF00E000BFB9
:1004F00000BF384601F056F9BDE8F0812DE9F04122
:10050000044600250026A768D4F80C802046FFF793
:10051000CFFDBDE8F08100002DE9F84F064600BF91
:1005200006F5337000F005FC0028F9D14FF4807017
:10053000FFF77DFD04460025002756E04FF0000838
:10054000394606F5337000F06FFC8046B8F1000FB5
:100550004AD038E00020605500BF11E0691E091A3A
:100560000DD4691E091A615C0D2904D0691E091A8F
:10057000615C0A2903D10022691E091A6254401CD9
:100580000328EBDBD6F8AC0DE8B14FF48070FFF731
:100590004EFD8246B8F8062017A15046FFF78DFDA4
:1005A0005046FFF74EFD00EB0A0B59462046FFF779
:1005B00089FD52467221D6F8AC0DFFF74CFD50462E
:1005C000FFF744FD00BF0A200090B8F8061064232E
:1005D000224606F5337000F0ACFC05460DB1012053
:1005E00000E000200028B5D17F1C052FA6DB2046A7
:1005F000FFF72CFDBDE8F88F25643A002DE9FE4F8A
:100600000446A668E56804F5337000F0AAFC04F51A
:10061000337000F0D7FC70B941F2883065A367A24F
:100620006BA100902046FFF7FDFC2046D4F8D010C7
:100630008847BDE8FE8F94F8C00131287CD10120A5
:10064000C4F8C40104F5337000F0B4FD2346624AD7
:100650007A4462A12046FFF73AFD06EB46082F4692
:100660002D205A21CDE90010E81705EB907083107A
:100670004FEAE87008EB9070821000212046FFF7E7
:1006800008FDC4F8B40D5AA1D4F8B40DFFF706FD67
:1006900006EB460805EB45072D208221CDE9001029
:1006A000F81707EB907083104FEAE87008EB907032
:1006B000821000212046FFF7ECFCC4F8B80D4EA1D3
:1006C000D4F8B80DFFF7EAFC06EB4600052190FBD5
:1006D000F1FA2F464FEA45084FEAE87008EB9070B0
:1006E0008010E91705EB9171891014230022CDE9E0
:1006F000001A029004F5E4712046FFF7C5FCC4F827
:10070000A40D002712E004F5E47050F82780803033
:1007100050F82700007818B104F5127050F82780BF
:100720004146D4F8A40DFFF7D7FC7F1CD4F8C802CB
:10073000B842E8DC39E0FFE794F8C001322834D150
:100740000220C4F8C401B04605EB45072D208221E4
:10075000CDE90010F81707EB9070831006EBD87006
:10076000421000212046FFF794FCC4F8B80D22A1E6
:10077000D4F8B80DFFF792FCB2462F46B346A84610
:10078000E81705EB90708010009006EBDB704310CB
:10079000E81705EB90708210F01706EB907081104F
:1007A0002046FFF767FCC4F8A80D2046FFF77BFC46
:1007B00000BF3EE7C8B7B6A800000000C0B6D1C071
:1007C000C4A3BFE9B8B4CEBBCAA7B0DCA3A10000E4
:1007D000B4EDCEF300000000F50F0000D5FDD4DA33
:1007E000C9A8C3E8C0B6D1C0B4D3BBFA2E2E2E0020
:1007F000C1ACBDD300000000CFC2D2BBB2BD00006F
:100800007CB50446002611A012A314A216A10090E4
:100810002046FFF766FC08B9312600E03226D4E90D
:10082000020100231A46CDE900011946204600F0D6
:100830001FF8054685F8C06104F13C012846FFF722
:1008400055FC2846FFF757FC28467CBDB4D3BBFABD
:1008500000000000D6F7BBFA00000000C7EBD1A1F2
:10086000D4F1BDC7C9AB0000CCE1CABE0000000096
:100870002DE9FE4F07460E4690469A46DDF830B009
:100880000EB9254E7E4440F6C450FFF7D0FB044617
:10089000002C39D040F6C45200212046FFF730FC2E
:1008A0000D98434632463946CDE900AB02902046CA
:1008B000FFF72BFC20B92046FFF7C8FB002423E0FC
:1008C00016A060610120606618487844C4F8D00022
:1008D0000020A063164860631020FFF71BFCC4F8DB
:1008E000BC0100250EE01420FFF7A1FB04F5E47124
:1008F00041F825001420FFF79AFB04F5127141F826
:1009000025006D1C202DEEDB00F068FF09484844EF
:1009100004602046BDE8FE8FC5FBFFFF57494E5FD0
:100920004368617453747275637400006B00000057
:10093000ACC1D7000800000070B5044600F00AFF03
:10094000064600250CE004F5E47151F82500FFF798
:100950007DFB04F5127151F82500FFF777FB6D1C44
:10096000202DF0DB04F5337000F02CFBD4F8BC0133
:10097000FFF7D0FB2046FFF7D2FB00200449494493
:10098000086000F015FF304600F00CFF70BD00005D
:100990000800000070B5054600F0DCFE044607487C
:1009A0004844006820B1054848440068FFF7C4FF88
:1009B000204600F0F7FE002070BD00000800000097
:1009C0000146FF20302904DB392902DCA1F1300285
:1009D000D0B2412904DB462902DCA1F13702D0B2B2
:1009E000704710B500F062FC002010BD2DE9F04DFD
:1009F00004460E4617469846DDE908AB2078FF28E6
:100A000003D04FF0FF30BDE8F08D701E205CFC2855
:100A100002D04FF0FF30F6E74FF0FF35721EFB219A
:100A2000601C00F002FE0546681C30B3BAF1000FEE
:100A300002D0FB208AF80000B8F1000F05D029464B
:100A4000601C00F011FFC8F800000FB1601C386096
:100A50000A9840B1F21E511B621C2A44501C00F03F
:100A600003FF0A990860BBF1000F04D0601C284402
:100A7000401CCBF800000020C5E7721EFA21601C64
:100A800000F0D3FD0546681C30B3BAF1000F02D068
:100A9000FA208AF80000B8F1000F05D02946601C42
:100AA00000F0E2FEC8F800000FB1601C38600A9840
:100AB00040B1F21E511B621C2A44501C00F0D4FEAF
:100AC0000A990860BBF1000F04D0601C2844401C48
:100AD000CBF80000002096E74FF0FF3093E7F8B521
:100AE000054600200090002400260EE09DF800003E
:100AF000FF2800D101261EB19DF800002855641C76
:100B00009DF80000FC2800D104E0684600F0E2FBFC
:100B10000028EBD000BF9DF80000FC2801D1204642
:100B2000F8BD4FF0FF30FBE710B500F0DDFB002013
:100B300010BD70B505460E46002403E0285D00F0A8
:100B400047FC641CB442F9DB002070BD2DE9F04184
:100B500005460C461646FF201349494408700846CE
:100B60004570FD20887004B14EB9FC200E494944FF
:100B7000C87004210C484844FFF7DBFF11E03246FF
:100B800009494944C91C204600F035FD0746FC21AF
:100B9000F81C054A4A441154391D1046FFF7C9FF95
:100BA00000BF0020BDE8F0814C0200002DE9F047B5
:100BB00006460F463546B8460024A24617E0287878
:100BC000FFF7FEFE8246BAF1FF0F0FD008EB64007C
:100BD000007804F0010109B1002100E004210AFAC3
:100BE00001F1084308EB64010870641C6D1C28784F
:100BF0000028E4D12046BDE8F08730B502460B4618
:100C00000BB9002030BD002418E0C4EB041000EB49
:100C1000C00502F1080000EB8501C88868B9D2F868
:100C2000B45A0D60B2F8B80A8880CB800120886081
:100C30005068401C50600120E4E7641C052CE4DB94
:100C40000020DFE72DE9F04D04468B461746984615
:100C5000DDF824A000BFD4F8B00A01280EDAD4F8D9
:100C6000B00A00EBC00101EB001104F694200D184E
:100C7000D4F8B00A401CC4F8B00A23E0D4F8B00A93
:100C8000401E00EBC00101EB001104F694200D188A
:100C9000002612E0721C02EBC20303EB021304F6FF
:100CA0009422991806EBC60202EB061304F694226E
:100CB00098181922FFF738FA761CD4F8B00A401EAB
:100CC000B042E7DC2F703A465946681CFFF72CFA11
:100CD000781C054485F800806D1C85F800A05246FC
:100CE000681C0899FFF720FA0120BDE8F08DF8B5DF
:100CF00004460D4604F6BA26002000900622294636
:100D00002120FFF723FF6A463146204600F0A4F871
:100D100001280CD13078012809D104F52860296810
:100D2000C4F8B41AA988A4F8B81A0120F8BD0020A4
:100D3000FCE730B5A1B005460024642108A8FFF700
:100D4000F8F908A8FFF7CBFE0446601C28B908A8EC
:100D5000FFF7F4F9002021B030BD00200790069085
:100D600005900490039006A807A903AA04ABCDE957
:100D70000021029005AA214608A8FFF737FE401C73
:100D800020B908A8FFF7DAF90020E4E79DF80C0085
:100D9000FB280BD1DDE90610CDE900019DF80C30F0
:100DA0002846DDE90421FFF74DFF1AE09DF80C000D
:100DB000FA2816D105980078012806D107984288AC
:100DC0000188284600F0E9F80BE005980078022831
:100DD00007D10698831E07980188821C284600F0D8
:100DE00020F90120B7E710B502460B460BB90020E9
:100DF00010BD002114E0C1EB011000EBC00402F1B2
:100E0000080000EB8400C088984208D1C1EB0110B3
:100E100000EBC00402F1080000EB8400E8E7491C85
:100E20000529E8DB0020E3E70246052912DAC1EBD9
:100E3000011000EBC00302F1080000EB8300C08842
:100E400040B1C1EB011000EBC00302F1080000EB60
:100E5000830070470020FCE77CB506460C4615462B
:100E600000BF3046FFF765FF00231A46194630469B
:100E7000CDE9004500F004F80028F2D001207CBD47
:100E80002DE9F04D05460F4690469A46DDF820B014
:100E9000D5F8B00A00284AD005F6942427B1227864
:100EA000611C3846FFF740F9B8F1000F02D02078F6
:100EB000C8F80000BAF1000F04D02078401C205C74
:100EC0008AF80000BBF1000F08D02078801C225C5B
:100ED0002078C01C01195846FFF726F9099820B15F
:100EE0002078801C215C09980160002612E0721CA9
:100EF00002EBC20303EB021305F69422991806EBEA
:100F0000C60202EB061305F6942298181922FFF781
:100F10000BF9761CD5F8B00A401EB042E7DCD5F8D4
:100F2000B00A401EC5F8B00A0120BDE8F08D0020CF
:100F3000FBE72DE9F0470746884614461D46DDF8D5
:100F400020A041463846FFF74EFF06463EB15346C5
:100F50002A462146304600F00EFBBDE8F08700200F
:100F6000FBE770B50446FFF7DFFD69202070002025
:100F70006060C4F8B00A00250AE0C5EB051101EB7A
:100F8000C10204F1080101EB820000F0E7FA6D1CD8
:100F9000052DF2DBFFF725FD70BD70B505460E4649
:100FA0001446012C04D131462846FFF726FE07E0FF
:100FB00024B93146284600F050F901E0002070BD08
:100FC0000120FCE7FEB5044604F6BA250020029095
:100FD000642600BF002211460320FFF7B7FD022060
:100FE000FFF7B1F82046FFF7A4FE02A800231A4637
:100FF0001946CDE900502046FFF742FF029801282C
:1010000009D12878012806D16420FFF79CF8FFF762
:10101000E8FC0120FEBD3000A6F10106DAD100BFD8
:10102000F8E72DE9F0410746884614461D4641463B
:101030003846FFF7D8FE064636B12A4621463046E6
:1010400000F0C2FABDE8F0810020FBE72DE9F8438B
:1010500007460D46144607F6BA2600200090206089
:10106000002211462320FFF771FD40F6AC50FFF738
:101070006AF850E06A4631463846FFF7EDFE01282F
:1010800047D10098012806D13078012801D1BDE868
:10109000F8830020FBE7009807283CDB206800EB82
:1010A000C00000EB4000284431680160B1888180B5
:1010B000B07940B2216801EBC10101EB4101294443
:1010C00088710098072818DD0098A0F107082168AA
:1010D00001EBC10101EB41012944C81D4246F11D4C
:1010E000FFF722F80021206800EBC00000EB400071
:1010F0002844C01D00F8081007E00020216801EB1B
:10110000C10101EB41012944C8712068401C2060E5
:1011100001E00020BBE7ADE72DE9F84582460F4628
:1011200090461C460AF6BA2500200090002624E0CE
:101130002F7038126870142C01DD142600E026464A
:1011400032464146A81CFEF7EFFFB21C2946072095
:10115000FFF7FCFC6A4629465046FFF77DFE012852
:1011600007D12878012802D12CB9BDE8F8850020E4
:10117000FBE70020F9E7A41BB044002CD8D10020E5
:10118000F3E733B581B0054605F6BA240020009098
:10119000012202A90620FFF7D9FC6A46214628460B
:1011A000FFF75AFE012803D12078012800D13EBD67
:1011B0000020FCE738B5044604F6BA25002000906C
:1011C000002211462020FFF7C1FC6A46294620462E
:1011D000FFF742FE012806D12878012803D16820B4
:1011E0002070012038BD0020FCE7F8B504460D460C
:1011F00004F6BA26002000902846FEF722FF074694
:101200003A4629460120FFF7A1FC6A4631462046AE
:10121000FFF722FE012803D13078012800D1F8BD64
:101220000020FCE738B5044604F6BA2500200090FB
:10123000002211461020FFF789FC6A462946204605
:10124000FFF70AFE012806D12878012803D1732070
:101250002070012038BD0020FCE72DE9F041054653
:101260000E4616B90020BDE8F081002719E0C7EB53
:10127000071000EBC00105F1080000EB8104E088D5
:10128000B0420DD10020E080A0602060A08004F179
:101290000C0000F0AFF86868401E68600120E2E7CB
:1012A0007F1C052FE3DB0020DDE7000010B5FEF713
:1012B0004FFF044600200649494448608860C860E2
:1012C000086148612046FEF748FF002010BD00007D
:1012D0003400000010B5044621460248484400F09E
:1012E000B0F810BD3400000000B587B001210846F9
:1012F000FEF738FF01211020FEF739FF07220921F0
:101300002F48FEF739FF07220A212D48FEF734FF48
:1013100000208DF81A0001208DF81B0002208DF8A6
:1013200018000002059002208DF8190005A9244834
:10133000FEF727FF00208DF81A0002208DF8180014
:101340004002059005A91E48FEF71BFF1D48FEF749
:101350001DFF4FF4E13001900020ADF80800ADF81A
:101360000A00ADF80C00ADF810000C20ADF80E002E
:1013700001A91448FEF70FFF01211248FEF710FFE4
:10138000114979442520FEF710FF012240F2255132
:101390000C48FEF70FFF25208DF8000000208DF887
:1013A000010001208DF802008DF803006846FEF769
:1013B00006FF4FF4007005494944086007B000BDBE
:1013C000000002400010014017050000340000003A
:1013D00010B5044621460648FEF7F6FE00BF802100
:1013E0000348FEF7F6FE0028F9D0002010BD0000EB
:1013F000001001400146002048608860C8607047C6
:1014000030B502460B46916854680BE002F11000BB
:10141000405C984201D1012030BD491C10688842CF
:1014200000DC00212000A4F10104EFD100BFF3E7AC
:1014300010B504464FF4007020602046FFF7DAFF35
:1014400010BD2DE9F04104460D464FF0FF36FEF782
:101450007FFE07462069C8B16068B8B104F1180082
:10146000A168405C28706068401E60602878FC2895
:1014700002D12069401E2061A068401CA060216844
:10148000A068884201DB0020A06000263846FEF7F5
:1014900064FE3046BDE8F0810246506890B102F12A
:1014A00010009368C05C08705068401E50609068DF
:1014B000401C906013689068984201DB00209060A7
:1014C000012070470020FCE72DE9F04104460D465D
:1014D0004FF0FF36FEF73CFE0746FF2D01D10120FD
:1014E0006061D4E90010884219DA6069B8B104F18A
:1014F0001800E16845546068401C6060FC2D04D110
:101500002069401C206100206061E068401CE060B0
:101510002168E068884201DB0020E0600026384650
:10152000FEF71BFE3046BDE8F0810246D2E90030EE
:10153000984211DA02F11000D368C1545068401C7F
:101540005060D068401CD0601368D068984201DBBE
:101550000020D060012070470020FCE710B5044651
:101560000020E080A0602060A08004F10C00FFF764
:101570005FFF012010BD2DE9F84305468846164659
:101580001F46394605F10C00FFF73AFF10B900205D
:10159000BDE8F88300240020009014E0694605F1BE
:1015A0000C00FFF779FF08B92046F1E72EB19DF84E
:1015B000000008F80400761E641C9DF80000B84284
:1015C00001D12046E4E7E9E72DE9F04105460E4662
:1015D0001746002409E0315D05F10C00FFF7A5FF77
:1015E00010B92046BDE8F081641C3800A7F101075E
:1015F000F1D12046F6E730B503460C460FE01878E7
:10160000F02804DA18780870491C5B1C07E0F02009
:101610000870491C1878F0380870491C5B1C1000D1
:10162000A2F10102EBD1081B30BD10B5034600202A
:1016300004E01C5C8C4200D110BD401C9042F8DBE1
:101640004FF0FF30F8E700002DE9FF4D074600F0AE
:1016500081F883463E464FF45870FEF7E8FC054695
:1016600006F532722946101DFFF7F0FC002455E004
:1016700006F5E47050F8248004EBC40000EB400051
:101680002844407904EBC40101EB41012944097964
:1016900004EBC40202EB42022A44D27804EBC403F6
:1016A00003EB43032B449B78CDE90032CDE90210D4
:1016B00004EBC40000EB40002844437804EBC40072
:1016C00000EB40002A5C1CA14046FEF7F6FC04EB50
:1016D000C40000EB40002844C079C0B106F5127088
:1016E00050F8248004EBC40101EB41012944C81DDA
:1016F000FEF7A7FC00F1010A04EBC40000EB400078
:101700002844C11D52464046FEF768FD05E0002111
:1017100006F5127050F824000170641CD6F8C80257
:10172000A042A5DC2846FEF791FC584600F03AF8A6
:10173000002004B0BDE8F08D2530325825303258F5
:10174000253032582530325825303258253032581D
:101750000000000010B5FEF746FD0446034878443B
:101760000068FEF745FD204610BD00008E01000018
:1017700070B50446FEF737FD05462946064878440D
:10178000FEF74EFC05484844046005487844034988
:1017900049440968486170BD6E0100000400000002
:1017A00005F2FFFF10B504462046FEF721FD10BDEF
:1017B00009484844006868B107484844006880699F
:1017C00040B10548484400688069401E02494944C8
:1017D000096888617047000004000000064848441A
:1017E000006840B10448484400688069401C0249D0
:1017F00049440968886170470400000070B50546D7
:101800002846FFF7B5FFFFF7E9FF002411A10020EC
:10181000FEF7F3FC04460CB9012000E0002068B19B
:101820000FA10020FEF7E9FC06463046FEF7E8FF70
:10183000044608A12046FEF7E5FC06E02146A06F1D
:10184000FEF7E5FC2046FEF756FCFFF7B1FF00204F
:1018500070BD0000626C6520636861740000000068
:10186000686F6D650000000030B503460C461946F0
:101870001A460FE00878F02805DA08781070521C34
:10188000491C641E06E008784D7828441070521CEC
:10189000891CA41E002CEDD1D01A30BD70B5FFF705
:1018A00059FF044600250F48008800F0200078B159
:1018B0000C488088C5B229460B484844FFF704FE0F
:1018C0000A4848440068401C08494944086005E04B
:1018D00004480088C5B203488088C5B22046FFF797
:1018E00061FF70BD001001403400000010000000D6
:1018F00000000000CDA8B5C03100CDA8B5C03200B1
:10190000CDA8B5C03300CDA8B5C03400CDA8B5C0B2
:101910003500000000000000000000000000000092
:081920000100000000000000BE
:04000005000017FDE3
:00000001FF
